:0200000480007A
:100000006F008004732F2034930F80006308FF0378
:10001000930F90006304FF03930FB0006300FF038E
:10002000130F000063040F0067000F00732F2034CC
:1000300063540F006F00400093E19153171F0000BD
:1000400023223FFC6FF09FFF93000000130100008C
:10005000930100001302000093020000130300004C
:100060009303000013040000930400001305000034
:10007000930500001306000093060000130700001C
:100080009307000013080000930800001309000004
:1000900093090000130A0000930A0000130B0000EC
:1000A000930B0000130C0000930C0000130D0000D4
:1000B000930D0000130E0000930E0000130F0000BC
:1000C000930F0000732540F16310050097020000B4
:1000D000938202017390523073500018970200000F
:1000E00093824202739052309B021000939252030B
:1000F0009382F2FF7390023B9302F0017390023AF5
:100100007350403097020000938242017390523046
:10011000735020307350303093010000970200007C
:10012000938282EE73905230130510001315F5017F
:10013000635C05000F00F00F930110009308D005D9
:10014000130500007300000093020000638A0200A0
:1001500073905210B7B200009B82921073902230BD
:100160007350003097020000938242017390123462
:10017000732540F1730020309300000013870000C6
:10018000930300009301200063127728930010006E
:100190001387100093032000930130006318772623
:1001A00093003000138770009303A0009301400078
:1001B000631E772493000000138700809303008060
:1001C0009301500063147724B70000801387000068
:1001D000B703008093016000631A7722B7000080A4
:1001E000138700809B03F0FF9393F30193830380B5
:1001F00093017000631C7720930000001387F07F49
:100200009303F07F9301800063127720B700008092
:100210009B80F0FF13870000B70300809B83F3FFF0
:10022000930190006314771EB70000809B80F0FF5D
:100230001387F07F9B0310009393F3019383E37F75
:100240009301A0006314771CB70000801387F07F30
:10025000B70300809B83F37F9301B0006318771A84
:10026000B70000809B80F0FF13870080B7F3FF7F0B
:100270009B83F37F9301C000631A771893000000FB
:100280001387F0FF9303F0FF9301D00063107718FA
:100290009300F0FF13871000930300009301E00028
:1002A000631677169300F0FF1387F0FF9303E0FFC8
:1002B0009301F000631C7714B70000809B80F0FF6F
:1002C000138710009B0310009393F3019301000127
:1002D000631E77129300D0009380B00093038001D7
:1002E0009301100163947012130200009300D00078
:1002F0001387B000130307001302120093022000BB
:10030000E31652FE930380019301200163107310E2
:10031000130200009300D0001387A0001300000018
:10032000130307001302120093022000E31452FE8D
:100330009303700193013001631A730C13020000E0
:100340009300D000138790001300000013000000FA
:10035000130307001302120093022000E31252FE5F
:1003600093036001930140016312730A13020000BA
:100370009300D0001387B0001302120093022000F4
:10038000E31852FE93038001930150016310770834
:10039000130200009300D000130000001387A00098
:1003A0001302120093022000E31652FE9303700121
:1003B00093016001631C7704130200009300D000D6
:1003C00013000000130000001387900013021200B6
:1003D00093022000E31452FE930360019301700125
:1003E00063167702930000029303000293018001D9
:1003F000639E70009300100213802003930300009B
:100400009301900163147000631030020F00F00F2D
:10041000638001009391110093E111009308D005CE
:1004200013850100730000000F00F00F930110000E
:100430009308D0051305000073000000731000C07E
:1004400000000000000000000000000000000000AC
:10045000000000000000000000000000000000009C
:10046000000000000000000000000000000000008C
:0C04700000000000000000000000000080
:1010000000000000000000000000000000000000E0
:1010100000000000000000000000000000000000D0
:1010200000000000000000000000000000000000C0
:1010300000000000000000000000000000000000B0
:081040000000000000000000A8
:040000058000000077
:00000001FF
